:10000000000008308A000F2FFF00030E8312031335
:10001000A1000A08A0008A010408A2007708A30032
:100020007808A4007908A5007A08A6007B08A70034
:10003000831383128B1E1E280B193128220884007B
:100040002308F7002408F8002508F9002608FA001C
:100050002708FB0020088A00210E8300FF0E7F0E78
:1000600009008A110A1273290A108A100A118207DC
:100070006D346F3474346F3472345F3463346F347E
:1000800075346E347434733420343D342034253464
:100090006C3464340D340A3400340A108A100A11A6
:1000A00082070A3400340A108A100A118207453484
:1000B00052345234203425343234583425343234D6
:1000C00058340D3400340A108A100A118207523451
:1000D000443459340D3400340A108A100A1182074E
:1000E000533454344F3450345F3450344F345334D9
:1000F000203425346C3464340D3400340A108A10F2
:100100000A1182075334543441345434553453342F
:1001100020343034783425343034323458340D348B
:1001200000340A108A100A11820750344F345334B5
:100130004934543449344F344E34203425346C34EB
:1001400064340D3400340A108A100A1182072034F6
:1001500000340A108A100A1182074F345034453493
:100160004E3400340A108A100A11820743344C348A
:100170004F345334453400340A108A100A11820770
:100180004D344F345634453400340A108A100A1165
:1001900082075334453454345F34533454344F3429
:1001A000503400340A108A100A118207473445344B
:1001B00054345F34533454344F34503400340A10C0
:1001C0008A100A1182074A344F3447345F344F345F
:1001D00000340A108A100A1182074A344F34473417
:1001E0005F34433400340A108A100A1182074734FE
:1001F000453454345F3450344F34533400340A148B
:100200008A100A1182074734453454345F3453341A
:1002100054344134543400340A148A100A118207C9
:100220004534433448344F3400340A148A100A11D8
:10023000820743344C3452345F3450344F34533497
:1002400000340A148A100A118207533448344F3498
:1002500057345F3443344E345434533400348316AB
:100260003E0840068039C200BE1B382983123E2951
:10027000BD09BE09BD0A0319BE0A83128316C01B3D
:10028000432983124929BF09C009BF0A0319C00ABB
:1002900083121030F700FA018316C101831283160E
:1002A000BE0CBD0C0318562983125D293F08FA07BE
:1002B0000318C10A4008C10783128316C10CFA0C47
:1002C000F90CF80CF70B6529672983124F29C21B1B
:1002D0006B2983127129F809F909F80A0319F90A37
:1002E000831200000034891083168910FF308800C3
:1002F0008312310808028316BC0083128914831606
:1003000089103C088039003A031D882983129C29F2
:10031000831283163C08FF3A013E8312B10200307B
:10032000031C0130B2020030031C0130B302003064
:10033000031C0130B402AC2983163C088312B107B8
:10034000003003180130B207003003180130B30742
:10035000003003180130B407FA0183163C08F70097
:10036000F71BFA038312B5007A08B6003608831625
:10037000BE00831235088316BD00C0013D30BF00AA
:1003800083122F217908B6007808B500B70A03193F
:10039000B80A0B118A110A121E288B128101B801AA
:1003A000B7018B1600348B120911831609118312C1
:1003B0000915831609118312B401B301B201B10109
:1003C0008B160034E801831686148312861C681489
:1003D000831606168312061EE814831686168312E9
:1003E000861E6815B008031DE8156808F80000347B
:1003F00003178D018F0183168C130C1483120C08C4
:100400000313C300013003178D008F0183168C1373
:100410000C1483120C080313C400023003178D0060
:100420008F0183168C130C1483120C080313C50060
:10043000033003178D008F0183168C130C14831265
:100440000C080313C6004308BE004408BD0045085D
:10045000BC004608BB00043003178D008F018316D3
:100460008C130C1483120C080313C30005300317FC
:100470008D008F0183168C130C1483120C08031348
:10048000C400063003178D008F0183168C130C14E3
:1004900083120C080313C500073003178D008F016A
:1004A00083168C130C1483120C080313C600430824
:1004B000C2004408C1004508C0004608BF003F080C
:1004C0003B02031D722A40083C02031D722A4108A8
:1004D0003D02031D722A42083E02031D722A0130AA
:1004E000AF00732AAF013B08F7003C08F8003D0855
:1004F000F9003E08FA008A150A126A2F8C1E7E2A1D
:100500001808A8001A08F800A81C882A181218163B
:1005100000000034EA1B9D2A0F30F700690EF70532
:100520000A3077020318972A3030F707992A6A08A9
:10053000F70777080C1E9A2A99000F30E9050A3050
:1005400069020318A52A3030A72AEA136A08E907C6
:1005500069080C1EA92A99000034E2217808E700F6
:10056000E608031DB82A67080139003A0319D82A9A
:10057000E80168085320E80A0C1EBC2A99000430E0
:100580006802031DB92A6708E9003730EA008A22A9
:100590006608E9003730EA008A220D300C1ECE2AA8
:1005A0009900B9080319D82A0A300C1ED52A9900D7
:1005B000E80168086320E80A0C1EDC2A9900043070
:1005C0006802031DD92AB9080319EA2A0A300C1E49
:1005D000E72A99000034DC080319F02A5C08F12AA4
:1005E0002908DE005E08E0005D08E1006008E20026
:1005F0006208840080080319172B6108E300630870
:1006000084008008031D092B60086202F8001A2B81
:10061000132B620884000008E400630884000008CB
:1006200064020319152BE30AFF2AE20AF82A60087C
:100630006202F8007808DE075E0884008008031D67
:10064000282B29088400203080000030F8005C2B23
:100650005E08E0005D08E1006008E20062088400D6
:10066000800803194B2B6108E300630884008008AD
:100670000319492B620884000008E4006308840021
:1006800000086402031D472B6208F8004D2BE30AA3
:10069000352BE20A2E2B0030F8007808DF005F08C7
:1006A000840080080319582B5F0884008001DF0A4A
:1006B0005F08A9005E08F80000345C0884000008A8
:1006C000DE005D08840000085E020319A52B5C08AB
:1006D00084000008DF005F08403C0318732B5F08AC
:1006E0005A3C03187B2B5F08603C0318B12B5F0852
:1006F0007A3C031CB12B5D0884000008E000600810
:10070000403C0318872B60085A3C03188F2B600865
:10071000603C0318B12B60087A3C031CB12B5C08C9
:1007200084000008E1005D088400203000076102B9
:100730000319A52B5D0884000008E3005C08840011
:10074000203000076302031DB12B5C088400800881
:10075000031DAD2B0030F800BF2B5C08DC0ADD0A5E
:100760005D2B5C0884000008DE005D088400000842
:100770005E020318BD2BFF30BE2B0130F8000034A1
:10078000F701F801F901FA018316AE01AF01B001DA
:10079000B1012D082C042B042A04031DD12B831234
:1007A000132C831220308316B20083120310831699
:1007B000A60DA70DA80DA90DAE0DAF0DB00DB10D75
:1007C0002D0831020319E62B8312F52B2C08300279
:1007D0000319EC2B8312F52B2B082F020319F22B94
:1007E0008312F52B2A082E028312031C082C831671
:1007F0002A08AE022B08031C2B0FAF022C08031C87
:100800002C0FB0022D08031C2D0FB102031483120C
:10081000F70DF80DF90DFA0D8316B20B102C122CF2
:100820008312D62B83120000AE30840000340408FB
:100830008316A000F51B1E2C83122E2C2D30831244
:100840000C1E202C9900F209F309F409F509F20AAB
:100850000319F30A0319F40A0319F50A3B30831646
:10086000A5009A30A400CA30A300A2010A30A1005A
:10087000831275088316A9007408A8007308A700DE
:100880007208A6002508AD002408AC002308AB00C0
:100890002208AA008312C0230008F200840A00087C
:1008A000F300840A0008F400840A0008F500FD3013
:1008B0008407F708031D7A2C83162108013A031DCB
:1008C000632C83127A2C2008031D682C83127D2C44
:1008D0000F392102031D6E2C8312732C031C722C02
:1008E0008312832C8312F0308316201B0030F70014
:1008F00083127D2C8316A00183123030F70777080E
:100900000C1E802C990083162508A9002408A80035
:100910002308A7002208A600AD01AC01AB010A30F4
:10092000AA008312C0237A088316A5007908A400C0
:100930007808A3007708A200A10B9F2CA12C83129A
:10094000392C83120034EF0166083107EA003208BF
:10095000EB0067080318670FEB073308EC00680823
:100960000318680FEC073408ED0069080318690FD5
:10097000ED07B41FBE2CED1BC02CD62CED1BED2CAF
:1009800034086D02031CED2C031DD62C33086C02B9
:10099000031CED2C031DD62C32086B02031CED2C1E
:1009A000031DD62C6A0831020318ED2C0130EE002D
:1009B00007113A113A088316870083128714BA1078
:1009C0003A088316870083120516831605128312D0
:1009D0008512831685128312022DEE0107153A1136
:1009E0003A088316870083128710BA103A088316D4
:1009F000870083120512831605128312851683164B
:100A000085128312CD213608FA003508B61F112D44
:100A10003508003CF700FA013608031C360FFA02CD
:100A20007708F1007A08F200F21F172D1E2DF20848
:100A3000031D262D7108C73C031C262DB808031D75
:100A4000262D3708063C031C262D032D6E0B4E2D3C
:100A5000ED1F2D2DB41B2F2D442DB41B452D6D08DE
:100A60003402031C452D031D442D6C083302031C66
:100A7000452D031D442D6B083202031C452D031D1B
:100A8000442D31086A02031CB92D83160616831201
:100A9000061A4D2D0730EF00B92D732DB41F532DBD
:100AA000ED1B552D6A2DED1B6B2D34086D02031CBB
:100AB0006B2D031D6A2D33086C02031C6B2D031D67
:100AC0006A2D32086B02031C6B2D031D6A2D6A0808
:100AD0003102031CB92D831686168312861A732DD4
:100AE0000830EF00B92D8C1E792D7E220630EF00E4
:100AF000B92D3608FA003508B61F872D3508003C99
:100B0000F700FA013608031C360FFA027708F100E5
:100B10007A08F200F21F8D2D942DF208031D972DF7
:100B20007108C73C031C972D0930EF00B92DAA08A6
:100B30000319B82DF10171083420F10A0C1E9E2D05
:100B400099000F307102031D9B2D41308400340841
:100B5000F5003308F4003208F3003108F2001724DE
:100B60000D300C1EB12D99000A300C1EB52D9900C8
:100B7000262D07113A113A08831687008312871031
:100B8000BA103A08831687008312051283160512DD
:100B9000831285128316851283126F08F8000034C1
:100BA000DC01E22178080439003A0319DA2D01301A
:100BB000B000D321B008031DE12D0A30E600AD22BC
:100BC000122EAF08031DE82D0B30E600AD22122EC9
:100BD00031082B02DD002C08DE003208031C320F26
:100BE000DE022D08DF003308031C330FDF022E085E
:100BF000E0003408031C340FE0026008E9005F08DD
:100C0000E8005E08E7005D08E600A3247808DC0041
:100C10005C08073C031D0F2EE601AD22122E5C0876
:100C2000E600AD228A150A129F2D5D30840000086F
:100C30000319292E0130F800F701F70B1D2EF80BD0
:100C40001C2E4A30F700F70B232E00000000800B0B
:100C50001A2E8A110A12B52EDC01E2217808043915
:100C6000003A0319392E0130B000D321E601AD223C
:100C7000C22E07153A113A0883168700831287108F
:100C8000BA103A08831687008312051283160512DC
:100C900083128516831685128312CD213608FA0039
:100CA0003508B61F5C2E3508003CF700FA013608FF
:100CB000031C360FFA027708DD007A08DE00DE1F1B
:100CC000622E692EDE08031D712E5D08C73C031CD1
:100CD000712EB808031D712E3708063C031C712EB7
:100CE0004E2E8C1E772E7E220630DC009E2E831622
:100CF00086168312861A7F2E0830DC009E2E360858
:100D0000FA003508B61F8D2E3508003CF700FA01B1
:100D10003608031C360FFA027708DD007A08DE0079
:100D2000DE1F932E9A2EDE08031D9D2E5D08C73C04
:100D3000031C9D2E0930DC009E2E712E07113A11E6
:100D40003A088316870083128710BA103A08831670
:100D500087008312051283160512831285128316EB
:100D600085128312C830DD00152E5C08083C031D77
:100D7000BF2E0130B000D321E601AD22C22E5C08A7
:100D8000E600AD228A150A12BE2D0130E700E80107
:100D900066086807840080080319E52E6808E80AD9
:100DA000660784000008EA006A082B3C0319E42E59
:100DB0006A082D3C0319E42E6A082F3C0318E32E21
:100DC0006A08393C031CE701C82E6708F8000034A4
:100DD0006608E7006708840080080319F12EE70A17
:100DE000EA2E66086702F8000034EB01E9010A30D8
:100DF000EA00E801E7016B08EB0A660784000008D7
:100E0000EC006C082F3C0318092F6C08393C0318C0
:100E1000112F6C082B3C0319112F6C082D3C031D5E
:100E2000FB2E6C082D3C031D1E2F0130E9006B08C2
:100E3000EB0A660784000008EC00282F6C082B3CA6
:100E4000031D282F6B08EB0A660784000008EC00DE
:100E50006C082F3C0318DA2F6C08393C031CDA2F7E
:100E60006C08303C031D4B2F66086B07840000089C
:100E7000783C0319422F66086B0784000008583C31
:100E8000031D4B2F1030EA00EB0A6B08EB0A6607D4
:100E900084000008EC006A080A3C031D7F2F6C08E0
:100EA0002F3C03187E2F6C08393C031C7E2F8316C1
:100EB000BE010A30BD00831268088316C000831289
:100EC00067088316BF0083120B080B058B13A00065
:100ED0002F2120088B047908EE007808ED003030CF
:100EE0006C026D07E7006E08E8000318E80A6B085B
:100EF000EB0A660784000008EC004F2FDA2F6A081F
:100F0000103C031DDA2F6C08603C03188E2F6C0810
:100F10007A3C031C8E2F6C08DF398F2F6C08EC0095
:100F20002F3C0318972F6C08393C03189F2F6C082F
:100F3000403C0318DA2F6C08463C031CDA2F6C087F
:100F40002F3C0318BD2F6C08393C031CBD2F031028
:100F5000670DED00680DEE00ED0DEE0DED0DEE0DE3
:100F6000ED0DEE0DF030ED0530306C026D07E70051
:100F70006E08E8000318E80AD32F0310670DED0090
:100F8000680DEE00ED0DEE0DED0DEE0DED0DEE0D1F
:100F9000F030ED0541306C020A3E6D07E7006E0847
:100FA000E8000318E80A6B08EB0A660784000008EB
:100FB000EC00832F6A080A3C031DE52F690BE52F1F
:100FC000E709E809E70A0319E80A6708F80068086A
:100FD000F9000034B9080319EF2F0030F02F013069
:0C0FE000B900E601AD228A150A12BF2EEE
:1010000069086D068039F600E91F1128E609E7092D
:10101000E809E909E60A0319E70A0319E80A0319C6
:10102000E90AED1F1E28EA09EB09EC09ED09EA0AB5
:101030000319EB0A0319EC0A0319ED0A2030F50035
:10104000F101F201F301F4016908FA006808F900FE
:101050006708F8006608F7000310771C3D286A0847
:10106000F1076B0803186B0FF2076C0803186C0F7D
:10107000F3076D0803186D0FF407F40CF30CF20C72
:10108000F10CFA0CF90CF80CF70CF50B2C28F61FE8
:101090005428F709F809F909FA09F70A0319F80AAF
:1010A0000319F90A0319FA0A00346D087406803925
:1010B0008316A5008312ED1F6828EA09EB09EC09E5
:1010C000ED09EA0A0319EB0A0319EC0A0319ED0A00
:1010D000F41F7528F109F209F309F409F10A03195B
:1010E000F20A0319F30A0319F40AF701F801F901E6
:1010F000FA018316A001A101A201A30174087304DF
:1011000072047104031D86288312C82883122030BC
:101110008316A40083120310EA0DEB0DEC0DED0D08
:101120008316A00DA10DA20DA30D740823020319AF
:101130009B288312AA28730822020319A12883126C
:10114000AA28720821020319A7288312AA28710865
:1011500020028312031CBD2871088316A0027208A6
:10116000031C720FA1027308031C730FA202740800
:10117000031C740FA30203148312F70DF80DF90D6D
:10118000FA0D8316A40BC528C72883128B28831257
:1011900000008316A51BCE288312DA28F709F80968
:1011A000F909FA09F70A0319F80A0319F90A0319E0
:1011B000FA0A8312A030840000345C08E6008A1129
:1011C000C5268A15F808031DEB280230E6008A11AF
:1011D000AD228A1597295C08E6008A11E8268A154F
:1011E0007808053C0318FA280330E6008A11AD227E
:1011F0008A159729DC08031D03290430E6008A11AB
:10120000AD228A1597295C08E6008A11F5268A1511
:101210007808F7007908F800F901FA01F81F122997
:10122000F903FA037A08E1007908E0007808DF00A2
:101230007708DE005E08F7005F08F8006008F90034
:101240006108FA00E11F36295E08003CF700F8014A
:101250005F08031C5F0FF802F9016008031C600FB0
:10126000F902FA016108031C610FFA027A08E90029
:101270007908E8007808E7007708E600E91B5729B5
:10128000E908031D5129E808031D51296708023C9C
:1012900003185729FF3A031D51296608E83C031833
:1012A00057290530E6008A11AD228A159729E901F0
:1012B000E8010D30E7001130E6006108ED0060083C
:1012C000EC005F08EB005E08EA0000207A08E90005
:1012D0007908E8007808E7007708E6006908ED007B
:1012E0006808EC006708EB006608EA00F401F30107
:1012F0000330F200E830F10055207A08E500790863
:10130000E4007808E3007708E2006508E900640873
:10131000E8006308E7006208E6008A11A3248A1542
:101320007808DD005D08E6008A11AD228A158A156D
:101330000A12E62DB008031DA3290A30E6008A111F
:10134000AD228A15662B5C08E6008A11C5268A152F
:10135000F808031DB1290230E6008A11AD228A1572
:10136000662B5C08E6008A11E8268A157808053C99
:101370000318C0290330E6008A11AD228A15662BB6
:10138000DC08031DCC293408E4003308E3003208EC
:10139000E2003108E100112A5C08E6008A11F52616
:1013A0008A157808F7007908F800F901FA01F81FA2
:1013B000DB29F903FA037A08E0007908DF007808EE
:1013C000DE007708DD00E901E8010D30E7001130AB
:1013D000E6006008ED005F08EC005E08EB005D08C9
:1013E000EA0000207A08E8007908E7007808E600BB
:1013F0007708E5006808ED006708EC006608EB0078
:101400006508EA00F401F3010330F200E830F1006E
:1014100055207A08E4007908E3007808E2007708AC
:10142000E100E41F142A152A192AE401E301E2016C
:10143000E1016408E8006308E7006208E60061086B
:10144000E5006808E90003178D018F01031369089F
:1014500003178C0083168C130C15831203130B08CF
:10146000F7008B135530831603178D00AA308D00BB
:101470008C1483120313831603178C1C422A8312C5
:1014800003133B2A0C117708831203138B0467089C
:10149000E900013003178D008F010313690803175A
:1014A0008C0083168C130C15831203130B08F700A2
:1014B0008B135530831603178D00AA308D008C14C2
:1014C00083120313831603178C1C692A83120313D8
:1014D000622A0C117708831203138B046608E90053
:1014E000023003178D008F010313690803178C0066
:1014F00083168C130C15831203130B08F7008B1340
:101500005530831603178D00AA308D008C1483127A
:101510000313831603178C1C902A83120313892A42
:101520000C117708831203138B046508E90003305C
:1015300003178D008F010313690803178C008316AE
:101540008C130C15831203130B08F7008B13553003
:10155000831603178D00AA308D008C148312031399
:10156000831603178C1CB72A83120313B02A0C119D
:101570007708831203138B046808E900043003170B
:101580008D008F010313690803178C0083168C13D9
:101590000C15831203130B08F7008B1355308316B9
:1015A00003178D00AA308D008C1483120313831649
:1015B00003178C1CDE2A83120313D72A0C11770819
:1015C000831203138B046708E900053003178D00AD
:1015D0008F010313690803178C0083168C130C15F5
:1015E000831203130B08F7008B1355308316031770
:1015F0008D00AA308D008C148312031383160317F9
:101600008C1C052B83120313FE2A0C1177088312FE
:1016100003138B046608E900063003178D008F0161
:101620000313690803178C0083168C130C1583129F
:1016300003130B08F7008B135530831603178D0027
:10164000AA308D008C1483120313831603178C1C8D
:101650002C2B83120313252B0C11770883120313F1
:101660008B046508E900073003178D008F01031311
:10167000690803178C0083168C130C15831203134F
:101680000B08F7008B135530831603178D00AA3013
:101690008D008C1483120313831603178C1C532B99
:1016A000831203134C2B0C117708831203138B0442
:1016B0006408AE006308AD006208AC006108AB00CE
:1016C0000130AF00E6018A11AD228A158A150A128F
:1016D0000D2E2030EC00E801E901EA01EB0163087E
:1016E000FA006208F9006108F8006008F7000310CA
:1016F000771C882B6408E80765080318650FE9075D
:1017000066080318660FEA0767080318670FEB07F8
:10171000EB0CEA0CE90CE80CFA0CF90CF80CF70CE1
:10172000EC0B772B8A150A12A42B2E08E3002D0848
:10173000E2002C08E1002B08E000E701E60103309D
:10174000E500E830E400692B7A08E3007908E2005C
:101750007808E1007708E00063088316A900831287
:1017600062088316A800831261088316A7008312FB
:1017700060088316A600AD01AC010D30AB0011303E
:10178000AA0083128A11C0238A157A08DF0079081B
:10179000DE007808DD007708DC00E00160088A11CF
:1017A0006C208A15E00A0C1ED32B990009306002C8
:1017B000031DCE2B413084005F08F5005E08F40065
:1017C0005D08F3005C08F2008A1117248A150D30B9
:1017D0000C1EE82B9900B9080319F22B0A300C1ED5
:1017E000EF2B9900E6018A11AD228A158A150A129B
:1017F0002A2E5C0B082CE9010130E8008630E70056
:10180000A030E6008A11A3248A157808DD00152C83
:10181000FF30E900FE30E8007930E7006030E60094
:101820008A11A3248A157808DD005D08E6008A1174
:10183000AD228A1500340408E600E01F292C2D3063
:101840000C1E202C99008403DF09E009DF0A03192C
:10185000E00A600EF038E200E207E23EE300323ECA
:10186000E50060080F39E307E307E507E93EE40018
:10187000E407E4075F0E0F39E407E507E40DE50D23
:10188000E509E50D5F080F39E507E20D0730E100D6
:101890000A30E507E403031C492CE407E303031CB7
:1018A0004D2CE307E203031C512CE207E103031C68
:1018B000552C6130840007306605840765300402CA
:1018C0000319762C0008F700031D6C2C661A742C83
:1018D000E6196E2C20306F2C0830E6003030F70708
:1018E00077080C1E712C9900840A5E2C0008F70002
:1018F0003030F70777080C1E7B2C99008A150A12E6
:10190000C82CB008031D8A2C0A30E6008A11AD22CB
:101910008A15D72C3408E9003308E8003208E700BC
:101920003108E600ED01EC010330EB00E830EA009D
:1019300000207A08E1007908E0007808DF007708E5
:10194000DE006108ED006008EC005F08EB005E0857
:10195000EA00F401F3010D30F2001130F1005520DE
:101960007808DD007708DC00DE015E088A1191202E
:101970008A15DE0A0C1EBA2C990009305E02031D7E
:10198000B52C103084005D08E0005C08DF001B2CE3
:101990000D300C1EC92C9900B9080319D32C0A303C
:1019A0000C1ED02C9900E6018A11AD228A158A15E9
:1019B0000A12842E8A11E2218A157808DC00DD01E2
:1019C0005D088A117E208A15DD0A0C1EE52C99001F
:1019D00009305D02031DE02C5C08E9003730EA00A5
:1019E0008A118A228A150D300C1EF42C9900B90830
:1019F0000319FE2C0A300C1EFB2C9900E6018A11FB
:101A0000AD228A158A150A12A12EDD01DC015A3099
:101A100084005C0884075D088A11A3208A15800071
:101A200000380319162DDD0ADC0A072D3C30DC00D6
:101A30000F30DD00DD03DE018A117E228A15780871
:101A4000DF00083C031D382DDE080319372DDE03A7
:101A5000B9080319372D5F080C1E2C2D9900203072
:101A60000C1E302D99005F080C1E342D9900512D4D
:101A70005F081F3C0318512D5F087E3C031C512D4D
:101A80005D085E020318512D5E08DE0A5C078400C3
:101A90005F088000B9080319512D5F080C1E4E2DF8
:101AA00099005F080D3C031D1C2D5C085E07840037
:101AB0008001B9080319712DE00160088A114D20D9
:101AC0008A1500380319692DE00A0C1E652D99004E
:101AD0005D2D0D300C1E6A2D99000A300C1E6E2DE6
:101AE0009900BC08031D792DE6018A11AD228A15E3
:101AF0000C2F3C30DC005A30DD008A11EB228A15B5
:101B00007808BB00DD01DC014B3084005C088407F1
:101B10005D088A11A9208A15800000380319932DC9
:101B2000DD0ADC0A842D3B08DC004B30DD008A1125
:101B30005D238A15F808031DA12D8A11D02D8A1561
:101B40000C2FDD01DC014B3084005C0884075D084C
:101B50008A11B2208A15800000380319B22DDD0ADF
:101B6000DC0AA32D3B08DC004B30DD008A115D232D
:101B70008A15F808031DC02D8A112C2E8A150C2FEA
:101B8000DD01DC014B3084005C0884075D088A11AC
:101B9000BC208A15800000380319D12DDD0ADC0A2B
:101BA000C22D3B08DC004B30DD008A115D238A1515
:101BB000F808031DE72DDC015A30DD008A11EB2205
:101BC0008A157808BB003B08DC00DD280C2FDD01FE
:101BD000DC014B3084005C0884075D088A11C52055
:101BE0008A15800000380319F82DDD0ADC0AE92D7A
:101BF0003B08DC004B30DD008A115D238A15F808B4
:101C0000031D0E2EDC015A30DD008A11EB228A15ED
:101C10007808BB003B08DC009A290C2FDD01DC01B1
:101C20004B3084005C0884075D088A11D2208A1535
:101C30008000003803191F2EDD0ADC0A102E3B0835
:101C4000DC004B30DD008A115D238A15F808031D86
:101C50002B2E952B0C2FDD01DC014B3084005C0812
:101C600084075D088A11DF208A1580000038031977
:101C70003C2EDD0ADC0A2D2E3B08DC004B30DD005B
:101C80008A115D238A15F808031D4A2E0130DC00F5
:101C9000F9230C2FDD01DC014B3084005C08840744
:101CA0005D088A11E9208A158000003803195B2E2F
:101CB000DD0ADC0A4C2E3B08DC004B30DD008A11CB
:101CC0005D238A15F808031D682EDC01F9230C2F0B
:101CD000DD01DC014B3084005C0884075D088A115B
:101CE000F3208A15800000380319792EDD0ADC0AFA
:101CF0006A2E3B08DC004B30DD008A115D238A151B
:101D0000F808031D852E812C0C2FDD01DC014B30E2
:101D100084005C0884075D088A11FF208A15800012
:101D200000380319962EDD0ADC0A872E3B08DC00FA
:101D30004B30DD008A115D238A15F808031DA22EA1
:101D4000DA2C0C2FDD01DC014B3084005C088407A9
:101D50005D088A110C218A15800000380319B32E02
:101D6000DD0ADC0AA42E3B08DC004B30DD008A11C2
:101D70005D238A15F808031DC12E8A11EA2F8A15E2
:101D80000C2FDD01DC014B3084005C0884075D080A
:101D90008A1115218A15800000380319D22EDD0A18
:101DA000DC0AC32E3B08DC004B30DD008A115D23CA
:101DB0008A15F808031DE42E8A11D3218A15E6013D
:101DC0008A11AD228A150C2FDD01DC014B30840015
:101DD0005C0884075D088A1121218A15800000387B
:101DE0000319F52EDD0ADC0AE62E3B08DC004B3039
:101DF000DD008A115D238A15F808031D072FAA0844
:101E00000319042F0030052F0130AA000C2F0130D8
:101E1000E6008A11AD228A158A150A12772F8401ED
:101E20001F3083059F30840007308000A8011930DF
:101E30008316990026309800903083129800A901EB
:101E4000AA01AB01AC01AD01AE01AF01B001B5011A
:101E5000B601B701B801B901FF30BA0007113A1154
:101E60003A088316870083128710BA103A0883163F
:101E700087008312051283160512831285128316BA
:101E8000851283120530F700F71D4E2F07308101B0
:101E9000813084000008C0390F3880006400813030
:101EA00084000008C039770480008A11CD218A158A
:101EB0008A11D3218A158A11E2218A1578080439FA
:101EC000003A0319682F0130B0008A11D3218A1516
:101ED0008A11F8298A157A08AE007908AD007808C9
:101EE000AC007708AB008B16C0308B04052D762F25
:021EF00063008D
:02400E00B137C8
:00000001FF
